S12302007E02A300FF01FF010001010001FF01FF00FFFF2E2A4B424E454E53524C52504816
S1230220505444525348545053445442434F083505A80AEF0BB2080E0E3805790CD00CA977
S12302400F270E80BDC00308A600810426F639860DBDC003860A7EC0038DF420EB364444A0
S123026044448D02323936840F8A30813923028B07BDC003323936862020F637B6010D0C20
S1230280490C49BB010CF6010D0C59490C59490CFB010DB9010C0CCB198B36B7010CF7014C
S12302A00D3339CE0F47BD0259CE00206F00088C010C26F886FFCE00BCA700088C00FC26FD
S12302C0F8CE0F7FBD0259BDC006815327037C0055CE007CC640BD027B81FC230486042084
S12302E01981F723048603201181E023048602200981A02304860120014F7F00567D005569
S123030027169756BD027B81F023048603200981C02304860220014F9B56A7009B54975459
S1230320BD027B8438AA00A700085A27037E02D6BD027B840716BD027B84079721D7227CC3
S12303400020CE007CBD06E18640AA00A7008D32BD027B8B00199738BD027B847F8A238B93
S1230360001997378D3B7D00552705168D331B199739BD027B8407977ABD027B8407977B45
S1230380202A7F0057863097587F0059973C7F003D860F9746CE00616F00088C006A26F801
S12303A039BD027B840F8A318B001939BD027B84079747BD027B84079748BD06CBCE0F9F4A
S12303C0BD025996218D4EBD046A96228D47CE135DBD0259CE0075C603BDC006A700085ACA
S12303E026F7CE0FD7BD02598D31CE0FE8BD02598D3BCE0FFDBD02597F003196399732BDB6
S12304000549CE101FBD02598D4ACE1034BD02598D4D7E04798B31BDC00339DE37DF31BD48
S12304200549862EBDC0039628BD02663996547F00317F0032C60A10250C7C0032D13226E7
S1230440F67C003120EC1BD632585858581B9732BD05493996488DBD8D1096478DB7399689
S12304604A8DB28D0596498DAC39862DBDC00339DF319B329732DE31399639913B22037E74
S12304800D697D005426037E0D6E7D006F270CCE16BDBD0259BD0CBF7E0D76BD0D978602A5
S12304A0914E275F7F004E7D002627034A974EBD027B81FC230DCE14DBBD025986029766C9
S12304C0BD057EBD027B81FC2303BD0DCDBD0D197D00582A037E0D617D00792612967A91C4
S12304E047260C967B91482606CE1A11BD0259860391582302974E7D003C2A074F9757971E
S12305003C973DCE1040BD02597F00297F0078BDC006810D271616BDC006CE0218E100261C
S123052004A101270F08088C022E26F1CE18B3BD025920DB8616084A26FCEE00AD007D0024
S12305406C27037E0D767E04797F004D9631271384F027059631BD025D9631840FBD026636
S12305607C004D96327D004D260484F02703BD025D9632840FBD0266397D0057270A7F00FB
S123058057CE104BBD025939963C810123F97D006626EB7C0057CE003C860297317F003244
S12305A0BD0AD3CE106520DC7D0062270F7D00792604BD0E3139CE1A4DBD0259BD024F7F1A
S12305C00050964E81022603BD0382CE00FCDF33BD0674CE1187BD0248BD041BBD0674CE94
S12305E01194BD0248964E271A8101271181032705CE0FB62003CE11A2BD0248200ACE1175
S1230600AA20F6CE11B120F18D6ACE11B7BD0248BD04548D5FCE11C4BD0248BD045F8D5435
S1230620CE11D1BD0248DE58DF31BD05498D45CE11DCBD0248BD042D8D3ACE11E9BD024896
S1230640DE3CDF31BD05497D00572705CE0F9B2003CE0FBDBD02488D1BCE11F5BD02487F23
S1230660003196468B00199732BD0549DE73A600BD0B7C39BD024F860297307F004F8604C8
S12306809751DE33A6009756964A9150260D9649914F26078645BDC003200F9656CE0213A1
S12306A08403BD0470A600BDC003BD0276DE337C004F7A005127069656444420C908DF33D8
S12306C0A6007A003026B77C0050397F0026CE00FCC6104FA700085A26FACE007C9647D62A
S12306E04897565D27098608084A26FC5A26F796562704084A26FC7D002027047F00203990
S1230700DF73E600D7522736C407270AD730D726860297538D62D652C438270B545454D78D
S123072030860197538D51D652C540270A86019730860397538D41D6522A037C006FBD024A
S12307407B8407974BBD027B8407974CBD07C07D004D26EA964B9749964C974AD62658CE01
S1230760003E6F006F01BD027B8B00197F00319732BD0AD05A26EF39CE00FCBD027B840F2B
S1230780975ABD0470E600BD027B84039756270556564A26FBC50326DFDA539656270559F1
S12307A0594A26FBE7007A003026CD96538103260ED65A0C56965624028B049723D724392B
S12307C07F004DDF35CE00FC964C270508084A26FB964B81032303088004E60097562705CC
S12307E054544A26FBC4032710D74D7D002927097D00782607C1022703DE3539C6FC9656E1
S123080027060D59594A26FBE400E70020EB7D00652704BD0E31397D0046260ACE0FC3BD15
S123082002597C006B397C0078BD027B840F8A04972D7A00467F002A7F0025CE107DBD02FF
S123084059BD0A7B81072238BD0276BD0276972C7D00782620CE1097BD0259BD0A7B972D1C
S12308607D002B2607972A7D006126A7BDC006810D26F9962CCE020348BD0470962D26010B
S12308803997307D002A2704860F97309649D64AAB00EB01BD0A577D002E27037E092A7D6F
S12308A0002F27037E092A974BD74C7D00782705BD02768D1F7C0029BD07C0964D272B7D48
S12308C0007827037E0A1B810226037E09C4CE10AFBD0259964CBD0415BD046A964BBD04AE
S12308E0157D00782701397E09777D00782712964BD64C7A00302698CE1165BD02597E090F
S123090077964B9749964C974ABD027B8180230A8601BD0A988603BD0AC07A003027037E28
S1230920088C7D002A26037E09777D007827037E08F8962D97309647D6487D002A276EAB48
S123094000EB01974BD74CBD0A577D002E27037E09F77D002F27037E09F7964B9747964C3C
S123096097487C00258606BD0A988630BD0AC07A003026C2BD06CB7F004E96219147261C0D
S1230980D622D14826169623D6244C90498102220B5CD04AC10222048602974E7D006D27A1
S12309A003BD05A87D006E2703BD0AEF399B2EDB2F81072242C107223E9747D7488607BD94
S12309C00A9820B0CE10D4BD0259860197307F002A7C005B7A00547A00267C0078BD08D40E
S12309E0CE1774BD0259C66ABD0E04CE1382BD0259BD042D7E0901CE10F6BD025996604C64
S1230A008103260ACE1507BD02597C006C3997607D002526037E09777E0974CE114DBD0255
S1230A2059964D8102261A7A00267A00547C005BCE1344BD0248CE1382BD0259BD042D20B9
S1230A400D8101260A7C005CCE12FDBD024839CE13167C005D20F47F002E7F002F4D2A0523
S1230A607A002E2007810723037C002E5D2A047A002F39C10723037C002F394F972BBDC07E
S1230A8006812E27F781392207812F2303803039CE12ECBD024820E39B288109231F800AEE
S1230AA097287F003186019732DF35CE0037BD0AD0CE003ABD0AD0BD0DBDDE353997283959
S1230AC0DF35CE00587F00319732BD0AD3DE35390C200D8699903197318699903297320DE1
S1230AE0A601993219A701A600993119A700397D00632704BD0E31397F00427F00437F0014
S1230B00447F0045CE1202BD0259BD0454BD024F964726037C0044810726037C0045964896
S1230B2026037C0042810726037C0043DE7386F7BD04707D004227048D6820028D1886052A
S1230B40BD04708D118605BD04707D004327048D5120028D0139A6007D004427034F200252
S1230B608D1A8D1BA6008D148D15A6007D004527034F20028D068D07BD024F39A740391692
S1230B8084800C4949BD02661784404444BD025D17843848BD025D178407BD026608BD0246
S1230BA07639860397304F8DD67A003026F8BD024F397D00642704BD0E31397D0057270530
S1230BC0CE12152027CE1233BD0259DE58DF31BD0549CE124DBD0259BD0C6D9640915822FD
S1230BE008260D964191592307CE126BBD025939BD027B81F42308CE1289BD0259206396BB
S1230C0040913E2208264A9641913F23447F003E7F003FCE12A0BD0259CE1382BD0259D6B5
S1230C2026D75B9654109754BD042D7F0026CE00FC86109730C604A6004625124624010C55
S1230C405A26F646A700087A003026E920144620EFCE0040DF31CE003EBD0AD3CE12D1BDB1
S1230C600259DE40DF31CE0058BD0AD3397F00407F0041BDC006813025208D1F7D00272680
S1230C8011C6047800417900405A26F79B41974120E1CE12ECBD024820D9397F0027813972
S1230CA02203840F397C002739CE1422BD0259CE0075C603BDC006A100260E085A26F5CE98
S1230CC013F2BD02597C006C39CE1454BD0259398612913B22217D00702623BD027B81B003
S1230CE023037C0070BD027B8180221796219747962297487E0974CE147EBD025939CE17AD
S1230D008220F7BD027B84079747BD027B84079748CE14B1BD025920DB7D0026260139BD89
S1230D20027B81B0222DCE0071D62658BD0762DE71DF317D0057261CCE0058BD0AD3BD0205
S1230D404FDE71DF31BD0549CE13A1BD0248C6FABD0E0439CE003CBD0AD3CE13BDBD02592B
S1230D6039CE1574BD0259200DCE15AE20F6CE15DFBD02592008CE161CBD02592006CE16CF
S1230D8057BD0259CE1833BD0259BDC006815927037EC0007E02A3DE73A600905BD65C585B
S1230DA05858107D005D270B84BFC60AD721D7227F004EA7004F975B975C975D39CE00615B
S1230DC06D0027026A00088C006A26F439BD027B840716BD027B8407D75ACE007C7C002007
S1230DE0BD06E1E600C40796541097548680A700CE174ABD0259965ABD0415BD046A9656E4
S1230E00BD041539CE0061BD027B11230ABD027B84030DA900A700088C006A26EA7D006609
S1230E2027037F00577D006927067F006D7F006E39CE1782BD025939CE17BDBD0259CE1732
S1230E40D0DF33CE00616D002615DF5EDE330808080808080808080808DF33DE5E2019DFC9
S1230E605EDE33BD025908DF33DE5EC603BD02765A26FAA600BD042F088C006A26C820B7C0
S1230E807D00692704BD0E3139CE1A7EBD0259BDC00681542760814D272B815326EBCE1BBD
S1230EA077BD02597F006DBDC006815926037C006DCE1BA5BD02597F006EBDC0068159262E
S1230EC0037C006E39CE1B09BD0259CE00BCBD024F86089730A60081FF260DDF5ECE1B462C
S1230EE0BD0248DE5E082003BD0B7F7A003026E58C00FC26D9397D00652704BD0E31397F03
S1230F00006BCE1B4CBD0259BDC006813025F0271581392EEA840F976ABD08177A006A2743
S1230F20057D006B27F3397D00792614967A9147260E967B91482608CE18597C00792003B2
S1230F40CE1885BD0259390A2D202D202D202D202020532054204120522020205420522073
S1230F6045204B2020202D202D202D202D20202020202056455253494F4E20312E3204535B
S1230F80484F5254204F52204C4F4E472047414D453F2028532D4C293A20042055500453CF
S1230FA05441524241534520494E205155414452414E543A2004444F434B45440420444F35
S1230FC0574E04414C4C20544F525045444F5320464952454421040A495420495320535422
S1230FE04152444154452004544845204B4C494E474F4E53204E554D4245522004594F55A8
S1231000522054494D45204C494D49542028494E2053544152444154455329203D200459DF
S12310204F552041524520494E205155414452414E542004414E4420534543544F522004CE
S12310400A434F4D4D414E443F200454484520534849454C44532041524520444F574E2C97
S1231060205349520454484520534849454C4453204152452055502C205349520457484172
S12310805420434F555253452C205349523F2028302D37293A20045748415420574152509D
S12310A020464143544F522C205349523A200454484520454E5445525052495345204953F7
S12310C020424C4F434B454420415420534543544F52200457452756452052414D4D4544FB
S12310E02041204B4C494E474F4E20415420534543544F522004594F5527564520524541D9
S123110043484544205448452045444745204F46205448452047414C41585920414E4420D2
S1231120554E4B4E4F574E0D0A464F5243455320484156452053544F50504544205448451E
S123114020454E54455250524953452104594F555220544F525045444F204841532048490C
S1231160542041200454484520544F525045444F204841532052554E204F5554204F462076
S1231180454E4552475904202053544152444154453A20042020434F4E444954494F4E3A66
S12311A0200459454C4C4F57210452454421212104475245454E0420205155414452414E03
S12311C0543A20042020534543544F523A202020042020454E455247593A200420204B4C6C
S12311E0494E474F4E533A20042020534849454C44533A20042020544F525045444F533A2B
S123120020045343414E20464F52205155414452414E542004594F55204D555354204649C1
S1231220525354204C4F57455220534849454C4453210454484520415641494C41424C4535
S123124020454E455247592049533A2004484F57204D55434820454E455247592053484165
S12312604C4C2049205553453A2004594F5520444F4E2754204841564520454E4F5547485B
S123128020454E455247592104504841534F52532048415645204D4953464952454421043F
S12312A0414C4C204B4C494E474F4E5320494E205448495320534543544F52204841564589
S12312C0204245454E2044455354524F594544210454484520454E454D59204841532042FB
S12312E045454E2044414D414745440420494E56414C494420454E54525921200453544105
S1231300522C2042494C4C494F4E532048415645204449454404424153452C20594F55529B
S1231320204F4E4C5920534F55524345204F4620535550504C59204953204E4F5720474F0E
S12313404E4521044B4C494E474F4E2C20434F4E47524154554C4154494F4E5304454E540B
S1231360455220594F55522033204C45545445522041424F52542050415353574F52443ABB
S123138020045448452052454D41494E494E47204B4C494E474F4E53204E554D42455220FC
S12313A00420554E495420484954204F4E2054484520454E5445525052495345044B4C49FD
S12313C04E474F4E5320484156452041545441434B45442C204255542054484520534849A3
S12313E0454C44532041524520484F4C44494E472104454E54455250524953452048415382
S1231400204245454E2044455354524F594544202D20414C4C2048414E4453204C4F535485
S1231420210441424F52542053455155454E43452053544152544544202D2057484154209A
S123144057415320594F55522050415353574F52443F200441424F52542053455155454ECF
S12314604345204142414E444F4E4544202D2050415353574F5244204552524F520454481A
S1231480452054454C45504F52544552205245504149525320415245204E4F54205945548C
S12314A02046494E49534845442C20534F5252590454454C45504F52544552204D414C4689
S12314C0554E4354494F4E202D2042415345204E4F5420524541434845440407574527561F
S12314E0452048495420412053504143452053544F524D202D20534849454C4453204441DE
S12315004D4147454421045448452033524420415454454D505420544F204C4541564520CB
S12315205448452047414C415859204841532043415553454420414E0D0A4155544F4D4182
S12315405449432053454C462D44455354525543542053455155454E43452E2049542043FB
S1231560414E4E4F542042452053544F50504544212121040754484520454E544552505272
S1231580495345204953204F5554204F4620454E455247592E2049542043414E204E4F2039
S12315A04C4F4E4745522045584953542E0407594F5520484156452052554E204F555420EC
S12315C04F462053544152444154455320464F522054484953204D495353494F4E2E040ACA
S12315E007434F4E47524154554C4154494F4E53210A0D00000000594F55204841564520CA
S123160044455354524F59454420414C4C20544845204B4C494E474F4E532E04594F555213
S1231620204D495353494F4E205741532041204641494C5552452C2054484520464544456F
S1231640524154494F4E204D5553542053555252454E4445522E04544845204645444552DD
S12316604154494F4E20484153204245454E20534156454420425920594F55522047414C04
S12316804C414E5420414354494F4E532E0D0A594F55204152452041574152444544205420
S12316A048452053544152464C454554204D4544414C204F4620484F4E4F522E044D4553DA
S12316C0534147452046524F4D2053544152464C45455420434F4D4D414E443A0D0A202018
S12316E020202054484520454E544552505249534520484153204A555354204245454E20C8
S123170044455354524F59454420425920410D0A202020202053555045524E4F5641204913
S12317204E20495427532043555252454E54205155414452414E54202D20414C4C2048416E
S12317404E4453204C4F53542E040753454E534F5253205245504F5254204120535550451E
S123176052204E4F564120494E205155414452414E5420044241444C592044414D41474539
S123178044044445564943452049532044414D4147454420414E4420554E555341424C451C
S12317A02E2020524550414952532048415645204245454E2053544152544544040A444555
S12317C056494345202020202053544154555304454E47494E45532020200453484F525459
S12317E0205343414E044C4F4E47205343414E2004504841534F525320202004544F52503A
S123180045444F53202004534849454C44532020200454454C45504F5254455204545241F4
S123182043544F5220424D04434F4D5055544552202004574F554C4420594F55204C494B5E
S12318404520544F20504C415920414741494E3F2028592D4E293A200454484520534855D3
S123186054544C45204352414654204953205245504F52544544204F4E20424F4152442CE9
S123188020534952045448452053454E534F52532053484F57204E4F5448494E4720544FA9
S12318A0204245205049434B45442055502C205349520454484520434F4D4D414E44532037
S12318C041524520415320464F4C4C4F57533A0D0A0A434D4E44202020414354494F4E0D8A
S12318E00A20454E202020204143544956415445205741525020454E47494E47530D0A209A
S123190053522020202053484F52542052414E4745205343414E0D0A204C52202020204C9B
S12319204F4E472052414E4745205343414E0D0A205048202020204649524520504841532C
S12319404F52204245414D530D0A20505420202020464952452050484F544F4E20544F52CC
S12319605045444F530D0A2044522020202044414D414745205245504F52540D0A2053482E
S123198020202020534849454C4453205550204F5220444F574E0D0A20545020202020542A
S12319A0454C45504F525420544F2042415345205155414452414E540D0A2053442020205C
S12319C02053454C462044455354525543542053455155454E43450D0A2054422020202065
S12319E041435449564154452054524143544F52204245414D530D0A20434F202020204240
S1231A004154544C4520434F4D50555445520D0A0453454E534F5253205245504F52542055
S1231A2053485554544C452043524146542047414C494C4C454F20494E2054484953205100
S1231A4055414452414E542C205349520453485554544C452043524146542053454E534FD4
S1231A6052532050524F564944494E47204241434B5550205343414E2C2053495204434F00
S1231A804D50555445522049532043415041424C45204F4620332046554E4354494F4E53C0
S1231AA03A0D0A20202054203D20544F525045444F205350524541440D0A2020204D203D83
S1231AC0205052494E54205343414E20484953544F5259204D41500D0A20202053203D2079
S1231AE0534554204155544F205343414E0D0A0A454E54455220434F4D50555445522043C7
S1231B004F4D4D414E443A2004535441545553204F46205155414452414E54532057484537
S1231B204E204C415354205343414E4E454420282A2A2A2A203D204E4F205343414E20591B
S1231B404554290D0A042A2A2A2A2004454E544552204E554D424552204F4620544F525057
S1231B6045444F5320494E205350524541442028302D39293A20044155544F205343414EBD
S1231B80204F4E20464F522053484F52542052414E47452053454E534F52533F2028592DE6
S1231BA04E293A20044155544F205343414E204F4E20464F52204C4F4E472052414E47452D
S1151BC02053454E534F52533F2028592D4E293A2004E0
S9030000FC
